:100000000C9437080C9454080C9454080C9454081D
:100010000C9454080C9454080C9454080C945408F0
:100020000C9454080C9454080C9402150C94540825
:100030000C9454080C9473140C946C0F0C94540886
:100040000C9454080C9454080C94C2110C94F9119B
:100050000C9454080C9454080C9454080C945408B0
:100060000C9454080C945408496E76616C696420B1
:100070004D50335472696767657220536F756E64B3
:1000800020436F6D6D616E64001400D007D007D0FF
:1000900007D007D00700002C01E803E803E803E8D5
:1000A00003E80300009600D007D007D007D007D0A0
:1000B0000700000000FFFFFFFFFFFFFFFFFFFF0043
:1000C000001400D007D007D007D007D0070000E801
:1000D00003E803E803E803E803E80300009600D020
:1000E00007D007D007D007D00700000000FFFFFFB0
:1000F000FFFFFFFFFFFFFF00001E00D007D007D06B
:1001000007D007D00700001E00E803D007D007D0B3
:1001100007D00700001E00D007E803D007D007D0A3
:100120000700001E00D007D007E803D007D0070063
:10013000001E00D007D007D007E803D00700001E3C
:1001400000D007D007D007D007E80300001E00D07A
:1001500007D007D007D007D00700001E00D007D077
:1001600007D007D007D00700001E00D007D007D067
:1001700007D007D00700001E00D007D007D007D057
:1001800007D00700001E00D007D007D007D007D047
:100190000700001E00D007D007D007D007D0070007
:1001A000000000FFFFFFFFFFFFFFFFFFFF00000F4A
:1001B00000D007D007D007D007D00700000F00E815
:1001C00003D007D007D007D00700000F00D007E802
:1001D00003D007D007D00700000F00D007D007E8F2
:1001E00003D007D00700000F00D007D007D007E8E2
:1001F00003D00700000F00D007D007D007D007E8D2
:100200000300000F00D007D007D007D007D00700A9
:10021000000F00D007D007D007D007D00700000F8D
:1002200000D007D007D007D007D00700000F00D0BC
:1002300007D007D007D007D00700000F00D007D0A5
:1002400007D007D007D00700000F00D007D007D095
:1002500007D007D00700000F00D007D007D007D085
:1002600007D00700000F00D007D007D007D007D075
:100270000700000F00D007D007D007D007D0070035
:10028000000F00D007D007D007D007D00700000F1D
:1002900000D007D007D007D007D00700000F00D04C
:1002A00007D007D007D007E80300000F00D007D021
:1002B00007D007E803D00700000F00D007D007E8F9
:1002C00003D007D00700000F00D007E803D007D005
:1002D00007D00700000F00E803D007D007D007D0F1
:1002E0000700000F00D007D007D007D007D00700C5
:1002F000000000FFFFFFFFFFFFFFFFFFFF000014F4
:1003000000D007D007D007D007D00700001400E8BE
:1003100003D007D007D007D00700001400E803E897
:1003200003D007D007D00700001400E803E803E873
:1003300003D007D00700001400E803E803E803E84F
:1003400003D00700001400E803E803E803E803E82B
:100350000300001400E803E803E803E803E80300EF
:10036000001400E803E803E803E803E803000014CE
:1003700000E803E803E803E803E80300001400E8EA
:1003800003E803E803E803E80300005000E803E89B
:1003900003E803E803E80300001400D007E803E8DB
:1003A00003E803E80300001400D007D007E803E8DF
:1003B00003E80300001400D007D007D007E803E8E3
:1003C0000300001400D007D007D007D007E80300CF
:1003D000001400D007D007D007D007D007000014C2
:1003E00000D007D007D007D007D00700001400D0F6
:1003F00007D007D007D007D00700001400D007D0DF
:1004000007D007D007D00700001400D007D007D0CE
:1004100007D007D00700002800D007D007D007D0AA
:1004200007D00700000000FFFFFFFFFFFFFFFFFFF7
:10043000FF00001400D007D007D007D007D0070076
:10044000003200E803D007E803D007E803000032D9
:1004500000D007E803D007E803D00700003200E827
:1004600003D007E803D007E80300003200D007E814
:1004700003D007E803D00700003200E803D007E804
:1004800003D007E80300003200D007E803D007E8F4
:1004900003D00700003200E803D007E803D007E8E4
:1004A0000300003200D007E803D007E803D00700BC
:1004B000003200E803D007E803D007E80300003269
:1004C00000D007E803D007E803D00700003200E8B7
:1004D00003D007E803D007E80300003200D007E8A4
:1004E00003D007E803D00700003200E803D007E894
:1004F00003D007E80300003200D007E803D007E884
:1005000003D00700003200E803D007E803D007E873
:100510000300003200D007E803D007E803D007004B
:10052000003200E803D007E803D007E803000032F8
:1005300000D007E803D007E803D00700003200E846
:1005400003D007E803D007E80300003200D007E833
:1005500003D007E803D00700003200E803D007E823
:1005600003D007E80300003200D007E803D007E813
:1005700003D00700003200E803D007E803D007E803
:100580000300003200D007E803D007E803D00700DB
:10059000003200E803D007E803D007E80300003288
:1005A00000D007E803D007E803D00700003200E8D6
:1005B00003D007E803D007E80300003200D007E8C3
:1005C00003D007E803D00700003200E803D007E8B3
:1005D00003D007E80300003200D007E803D007E8A3
:1005E00003D00700006400D007D007D007D007D0A1
:1005F0000700000000FFFFFFFFFFFFFFFFFFFF00FE
:10060000001400D007D007D007D007D00700002D76
:1006100000D007D007D007D007D00700002D00D0AA
:1006200007D007D007D007D00700002D00D007D093
:1006300007D007D007D00700002D00D007D007D083
:1006400007D007D00700002D00D007D007D007D073
:1006500007D00700002D00D007D007D007D007D063
:100660000700002D00D007D007D007D007D0070023
:10067000002D00D007D007D007D007D00700002DED
:1006800000E803D007D007D007D00700002D00E80E
:1006900003E803D007D007D00700002D00E803E8E7
:1006A00003E803D007D00700002D00E803E803E8C3
:1006B00003E803D00700002D00D007E803E803E8B3
:1006C00003D00700002D00D007D007E803E803D0CF
:1006D0000700002D00D007D007D007E803D007009F
:1006E000002D00D007D007D007D007D00700002D7D
:1006F00000D007D007D007D007D00700002D00D0CA
:1007000007D007D007D007D00700002D00D007D0B2
:1007100007D007D007D00700002D00D007D007D0A2
:1007200007D007D00700002D00D007D007D007D092
:1007300007D00700002D00D007D007D007D007D082
:100740000700002D00D007D007D007D007D0070042
:10075000002D00D007D007D007D007D00700002D0C
:1007600000D007D007D007D007E80300002D00D045
:1007700007D007D007D007D00700002D00D007D042
:1007800007D007D007D00700002D00D007D007D032
:1007900007D007D00700002D00E803E803E803E8CE
:1007A00003E80300002D00D007E803E803E803E8AE
:1007B0000300002D00D007D007D007E803E80300AE
:1007C000002D00D007D007D007D007D00700002D9C
:1007D00000D007E803D007E803D00700002D00D0C1
:1007E00007D007D007D007D00700002D00E803D0BE
:1007F00007E803D007D00700002D00D007D007D0AE
:1008000007D007D00700002D00D007D007D007D0B1
:1008100007D00700002D00D007D007D007D007D0A1
:100820000700002D00D007D007D007D007D0070061
:10083000002D00D007D007D007D007D00700002D2B
:1008400000D007D007D007D007D00700002D00D078
:1008500007D007D007D007D00700002D00D007D061
:1008600007D007D007D00700002D00D007D007D051
:1008700007D007D00700002D00D007D007D007D041
:1008800007D00700002D00D007D007D007D007D031
:100890000700002D00E803D007E803D007E80300B5
:1008A000002D00D007D007D007D007D00700002DBB
:1008B00000D007D007D007D007D00700002D00D008
:1008C00007D007D007D007D00700002D00D007D0F1
:1008D00007D007D007D00700002D00D007D007D0E1
:1008E00007D007D00700002D00E803D007E803D0A9
:1008F00007E80300002D00D007E803D007E803D085
:100900000700002D00E803D007E803D007E8030044
:10091000002D00D007D007D007D007D00700002D4A
:1009200000E803E803D007D007D00700002D00D06F
:1009300007D007E803E803D00700002D00D007D058
:1009400007D007D007E80300002D00D007D007D05C
:1009500007D007D00700002D00E803E803D007D038
:1009600007E80300002D00D007D007E803E803D014
:100970000700002D00E803E803D007D007E80300D4
:10098000002D00D007D007D007D007D00700002DDA
:1009900000E803D007D007D007D00700002D00D013
:1009A00007D007D007D007D00700002D00D007E8F8
:1009B00003D007D007D00700002D00D007D007D004
:1009C00007D007D00700002D00E803E803E803D0B4
:1009D00007D00700002D00D007E803E803D007D0B8
:1009E0000700002D00D007D007E803D007D007008C
:1009F000002D00D007D007D007D007D00700002D6A
:100A000000D007D007D007D007D00700002D00D0B6
:100A100007D007D007D007D00700002D00D007D09F
:100A200007D007D007D00700002D00D007D007D08F
:100A300007D007D00700002D00D007D007D007D07F
:100A400007D00700002D00D007D007D007D007D06F
:100A50000700002D00D007D007D007D007D007002F
:100A6000002D00D007D007D007D007D00700002DF9
:100A700000E803D007E803D007E80300002D00D00A
:100A800007D007D007D007D00700002D00D007E817
:100A900003D007E803D00700002D00D007D007D00F
:100AA00007D007D00700002D00E803E803E803E8BB
:100AB00003E80300002D00D007D007D007D007D0EF
:100AC0000700002D00E803E803E803E803E803005B
:100AD000002D00D007D007D007D007D007000000B6
:100AE00000FFFFFFFFFFFFFFFFFFFF00006400D0DC
:100AF00007D007D007D007D00700000000FFFFFF96
:100B0000FFFFFFFFFFFFFF00000F00D007D007D05F
:100B100007D007D00700000F00E803D007D007D0A8
:100B200007D00700000F00D007E803D007D007D098
:100B30000700000F00D007D007E803D007D0070058
:100B4000000F00D007D007D007E803D00700000F40
:100B500000D007D007D007D007E80300000F00D06F
:100B600007D007D007D007D00700000F00D007D06C
:100B700007D007D007D00700000F00D007D007D05C
:100B800007D007D00700000F00D007D007D007D04C
:100B900007D00700000F00D007D007D007D007D03C
:100BA0000700000F00D007D007D007D007D00700FC
:100BB000000F00D007D007D007D007D00700000FE4
:100BC00000D007D007D007D007D00700000F00D013
:100BD00007D007D007D007D00700000F00D007D0FC
:100BE00007D007D007D00700000F00D007D007D0EC
:100BF00007D007D00700000F00D007D007D007D0DC
:100C000007E80300000F00D007D007D007E803D0A3
:100C10000700000F00D007D007E803D007D0070077
:100C2000000F00D007E803D007D007D00700000F5F
:100C300000E803D007D007D007D00700000F00D08E
:100C400007D007D007D007D0070000A08CFFFFFF18
:100C5000FFFFFFFFFFFFFF00009808FFFFFFFFFF00
:100C6000FFFFFFFFFF00000000FFFFFFFFFFFFFF90
:100C7000FFFFFF00004F4B0A0D000A0D4D534520AA
:100C8000436F6E74726F6C6C657220312E300A0D7A
:100C900000456E7465722061204D534520636F6D71
:100CA0006D616E64207374617274696E6720776918
:100CB000746820273A27200A0D000A0D73756172A7
:100CC000743120436F6D6D756E69636174696F6E09
:100CD000204F4B200A0D000A0D737561727432208B
:100CE000436F6D6D756E69636174696F6E204F4BF4
:100CF000200A0D002A2A556E7265636F676E697A45
:100D0000656420436F6D6D616E642053746172740D
:100D1000204368617261637465720D0A00446973EF
:100D2000706C6179696E673A0D0A00485020636FF4
:100D30006D6D616E640D0A00446973706C61792099
:100D4000636F6D6D616E640D0A00536F756E642084
:100D5000636F6D6D616E640D0A00416C74312063C8
:100D60006F6D6D616E642C206F7574707574207476
:100D70006F207375617274320D0A00416C743220F9
:100D8000636F6D6D616E642C20666F727761726443
:100D900020746F20736C617665206F6E20737561AF
:100DA00072740D0A002A2A496E76616C69642056B5
:100DB000464420436F6D6D616E640D0A0028436CDC
:100DC0006F736520616C6C2070616E656C73292097
:100DD0000D0A002853637265616D29200D0A0028F1
:100DE0005761766529200D0A0028466173742057E3
:100DF00061766529200D0A00284F70656E20436CCE
:100E00006F7365205761766529200D0A00284361BC
:100E10006E74696E61204D61726368696E6720410E
:100E20006E747329200D0A002853686F7274204372
:100E300069726375697429200D0A002843616E7414
:100E4000696E612044616E636529200D0A00284C9B
:100E5000656961204D65737361676529200D0A001E
:100E600028446973636F2044616E636529200D0A0D
:100E7000002853657420746F2051756965742920AA
:100E80000D0A002853657420746F2057696465202B
:100E90004177616B6529200D0A0028416C6C207038
:100EA00069652070616E656C7320746F20524329F0
:100EB000200D0A002853657420746F204177616B00
:100EC0006529200D0A002853657420746F20457829
:100ED000636974656429200D0A0028536372656193
:100EE0006D204E6F2050616E656C7329200D0A00D5
:100EF00028527974686D69632050616E656C73293E
:100F0000200D0A00284D61726368696E6720416E8A
:100F100074732050616E656C7329200D0A0000C245
:100F200001000100110011000C0000E100000A00A6
:100F30002500250021000096000019003900390025
:100F40003600127A00001F00460046004400807000
:100F5000000022004D004D004A00004B000036000A
:100F6000750075007200403800004A009C009C002B
:100F70009900802500007200EC00EC00E900C0122E
:100F80000000E900DA01DA01D70160090000D701A9
:100F9000B603B603B303B0040000B3036E076E07D5
:100FA0006B072C010000DC0EC11DC11DBE1D000021
:100FB000004180017900F13800001716800002021C
:100FC0000404662E6028008060000040040299112D
:100FD000100169115111F001A310F9100412F91157
:100FE000F111011000C002026100040444118911D2
:100FF000F811513989101139A910A810D910F80128
:1010000000281901AA02890098079A059911E81188
:101010009B11EA11F110003899018C029E0106061D
:1010200004060512891002041111060001000004D3
:10103000F811513989101139A910A810D910F801E7
:1010400000281901AA02890098079A059911E81148
:101050009B11EA11F110003899018C029E010606DD
:10106000040605122202100144040006FFFF1124A9
:101070001FBECFEFD8E0DEBFCDBF11E0A0E0B1E0F2
:10108000E2E7F9E302C005900D92A836B107D9F75F
:1010900015E0A8E6B1E001C01D92A034B107E1F768
:1010A0000E94440E0C94B71C0C9400001092AA01EC
:1010B0001092A90181E0809368010895109268015F
:1010C0001092AA011092A901089580EB94E09093E8
:1010D000AA018093A9018091680180937201109206
:1010E00068010895809172018093680108950E94BB
:1010F0005E1608951F93182F86E70E945E16812FB3
:101100000E945E161F91089584E6809300010E945C
:101110007A0808951092000180E00E947A080895EC
:101120008EEF809300010E947A08089582E38093F5
:1011300000010E947A08089520910001253630F4BC
:1011400084E690E0821B9109059724F484E680935D
:10115000000103C02B5F20930001809100010E94D9
:101160007A08089580910001882311F0853018F4E1
:101170001092000103C0855080930001809100010E
:101180000E947A0808951F93CF93DF93282F8A3007
:1011900008F04AC0882311F4162F40C06A3108F0C5
:1011A00043C06623E9F0282F30E0695189E190E0DF
:1011B000AC01249FC001259F900D349F900D1124F8
:1011C000162F180F675EF901EF5FFE4FE081D9011E
:1011D000A759BE4FE61710F4EC9320C06C931EC0C5
:1011E000853010F0E1E013C0A82FB0E0ED01C75941
:1011F000DE4F88818F5F8883FD01EF5FFE4F908116
:10120000981710F481E08883A759BE4FEC9189E1CB
:10121000289FC0011124182F19511E0F84E70E9426
:101220005E16812F0E945E16DF91CF911F91089567
:1012300080E06EEF0E94C308089580E06FEF0E9487
:10124000C308089561E070E080E090E023E330E0BF
:1012500040E050E00E942F18643110F481E012C089
:10126000962F9351933110F482E00BC0962F955234
:10127000983010F483E005C0962F9C52953028F4E6
:1012800084E0692F0E94C30808956053643018F405
:1012900085E00E94C3080895809168018823E1F0E9
:1012A0008091A9019091AA01892BB1F48091A901A3
:1012B0009091AA01892B81F40E94220968E572E0CD
:1012C00080E090E028EE33E040E050E00E942F18EC
:1012D0007093AA016093A90108951F93CF93DF93A0
:1012E000EC01DC010D900020E9F71197A81BB90B68
:1012F0008881843209F007C18A2F8250833008F038
:1013000002C11981812F90E0C0970A9790F4109242
:1013100068011092AA011092A901A33010F460E0B4
:1013200005C0CE0102960E949A19682F812F805322
:10133000E7C01235C9F11335F0F4163409F493C03F
:10134000173480F4133409F459C0143438F41B32C0
:1013500009F4B6C01D3209F0D6C0B5C0143409F086
:10136000D2C092C01D3409F4C3C01F3419F11C341B
:1013700009F0C9C028C0163609F4ABC0173650F4BE
:10138000173509F4ACC0133609F44BC0133509F016
:10139000BAC05AC0103709F49FC0133709F487C088
:1013A0001D3609F0B0C092C01092AA011092A90196
:1013B00081E021C0109268011092AA011092A90147
:1013C0000E949008A4C080EB94E09093AA018093BF
:1013D000A90180916801809372011092680187E0F1
:1013E00061E00E94C30880E391E19093AA01809399
:1013F000A901809172018093680189C080EB94E01B
:101400009093AA018093A901809168018093720151
:101410001092680188E065E00E94C30880EE95E1C3
:10142000E4CF80EB94E09093AA018093A90180918E
:101430006801809372011092680188E061E00E9467
:10144000C3088CE89AE0D1CF80EB94E09093AA0196
:101450008093A901809168018093720110926801C4
:1014600086E061E00EC080EB94E09093AA01809347
:10147000A90180916801809372011092680186E051
:1014800063E00E94C308B5CF80EB94E09093AA017B
:101490008093A90180916801809372011092680184
:1014A00088E066E00E94C30880EB9AE99ECF109224
:1014B00068011092AA011092A9010E94180927C080
:1014C0000E94B20824C00E949C0821C00E94960875
:1014D0001EC00E948A081BC00E94840818C0109277
:1014E00068011092AA011092A90188E062E008C088
:1014F000109268011092AA011092A90188E063E09D
:101500000E94C30804C088E690E00E945D12DF914B
:10151000CF911F910895E9E6F1E0119281E0E23761
:10152000F807D9F70E9496080E941D0989EA91E000
:101530000E94F50E0895FC01108275836483738305
:1015400062834183478346830895FC0190818181B2
:10155000981710F080E00895A481B5816D9387817C
:10156000815019F48181A81BB1098783B583A483B5
:101570009FB7F89480818F5F80839FBF81E008953B
:10158000FC0180818823E9F3A281B3812D918681BA
:10159000815019F48181A81BB109B383A28386838A
:1015A0009FB7F8948081815080839FBF822F0895D8
:1015B000FC018081882319F42FEF3FEF13C0A28133
:1015C000B3812D918681815019F48181A81BB109C5
:1015D000B383A28386839FB7F894808181508083F0
:1015E0009FBF30E0C9010895FC01808120E030E018
:1015F000882311F021E030E0C9010895CF93DF93F3
:10160000EC016AE071E00E94B819009739F485E7AF
:101610009CE00E945D1210927D017BC0CE016CE0C7
:1016200071E00E94B819009731F485E79CE00E94B0
:101630005D1281E067C0CE016EE071E00E94B819D2
:10164000009731F485E79CE00E945D1282E05AC069
:10165000CE0160E171E00E94B819009731F485E78E
:101660009CE00E945D1283E04DC0CE0162E171E01A
:101670000E94B819009731F485E79CE00E945D1242
:1016800084E040C0CE0164E171E00E94B819009787
:1016900031F485E79CE00E945D1285E033C0CE0105
:1016A00066E171E00E94B819009731F485E79CE08B
:1016B0000E945D1286E026C0CE0168E171E00E94C2
:1016C000B819009731F485E79CE00E945D1287E02D
:1016D00019C0CE016AE171E00E94B819009731F497
:1016E00085E79CE00E945D1288E00CC0CE016CE1B1
:1016F00071E00E94B819009741F485E79CE00E94D0
:101700005D1289E080937D0104C085EA9DE00E941E
:101710005D12DF91CF910895DF93CF9300D000D079
:1017200000D0CDB7DEB7FC0180818A3329F085EA8D
:101730009DE00E945D120EC0662311F480E301C09B
:10174000818189831A82CE010196BE016C5F7F4F31
:101750000E94FE0A26960FB6F894DEBF0FBECDBFDC
:10176000CF91DF9108950F931F938C018AE59DE03F
:101770000E945D12C8010E94D6158DE00E949A1544
:101780001F910F9108950F931F938C0188E39DE0A3
:101790000E945D12C8010E94D6158DE00E949A1524
:1017A0001F910F9108950F931F938C018BE29DE081
:1017B0000E945D12C8010E94D6158DE00E949A1504
:1017C0001F910F9108950F931F938C018AE59DE05F
:1017D0000E945D12C80101960E949A168DE00E9437
:1017E0005E161F910F9108950F931F938C018AE449
:1017F0009DE00E945D12C8010E946D091F910F912A
:1018000008958EE191E062E00E94F40B089581E278
:1018100091E062E00E94F40B08950F931F93DF9311
:10182000CF93CDB7DEB727970FB6F894DEBF0FBEC4
:10183000CDBF2DB73EB7285030400FB6F8943EBF0D
:101840000FBE2DBFEDB7FEB731968E010F5F1F4F54
:10185000ADB7BEB712961C930E93119724E231E0F8
:101860003383228384831582668317820E94DF1963
:10187000F80101900020E9F73197E01BF10B2DB73B
:101880003EB7285F3F4F0FB6F8943EBF0FBE2DBF47
:10189000C8016E2F0E94F40B27960FB6F894DEBF96
:1018A0000FBECDBFCF91DF911F910F9108950F9380
:1018B0001F938C0185E79CE00E945D1287EC91E00C
:1018C000B8010E94C1191F910F910895CF93DF9322
:1018D000EC018881DE010D900020E9F71197AC1B27
:1018E000BD0B6A2FAA2329F485E79CE00E945D12B4
:1018F00031C0853239F1863228F48132F1F08432F8
:1019000031F516C08A3329F0803469F08A32F9F44F
:1019100005C0CE016A2F0E948C0B1CC0CE016A2F1D
:101920000E94D30B17C0CE016A2F0E94C30B12C0B6
:10193000CE016A2F0E94F40B0DC0CE016A2F0E94C7
:10194000E30B08C0CE016A2F0E94B30B03C0CE0187
:101950000E94570CDF91CF91089520917E018D3028
:1019600071F4E22FF0E0E057FD4F108210927E01FB
:10197000CB0160E972E00E94C11981E00895E22F75
:10198000F0E0E057FD4F8083283C10F080E00895A0
:101990002F5F20937E0180E00895BC0110927D01AD
:1019A00087EC91E00E94C119109281010895EBEA41
:1019B000F1E08FEF9FEF8193919321E0ED3BF207F0
:1019C000D1F7CF0142970E94261708950F931F93D6
:1019D00008E513E0C80167EC71E049E050E00E94BF
:1019E000C819C8010E943D171F910F910895809159
:1019F000C5019091C601892B01F580917F01882353
:101A000059F088E593E067EC71E049E050E00E940E
:101A1000C81910927F010BC0E8E5F3E080E28193E2
:101A200093E0E136F907D9F781E080937F0181E205
:101A300090E09093C6018093C50188E593E00E94F1
:101A40003D170895E7ECF1E001900020E9F73197A8
:101A5000E75CF1402E2F109261038091C5019091B7
:101A6000C601892B59F481E290E09093C6018093DE
:101A7000C501809181018F5F809381016091810117
:101A8000693070F580E090E049E050E0461B510974
:101A900070E205C0FC01E85AFC4F70830196841780
:101AA0009507C4F389E0861BE82FFF27E7FDF09533
:101AB000E85AFC4F90E030E040E20FC0A92FBB276E
:101AC000A7FDB095A217B3072CF4A953BE4F8C9174
:101AD000808301C0408331969F5F961779F723C0BA
:101AE000422F50E09A01285F3F4F862F90E0281741
:101AF0003907BCF0962F9950E8E5F3E020E2A92FD2
:101B0000BB27A7FDB095A417B5072CF4A953BE4F6A
:101B10008C91808301C020839F5F3196961779F75F
:101B200002C01092810188E593E00E943D1708955C
:101B30008091C5019091C601892B09F580918001A2
:101B4000882361F0A8E5B3E0ECE2F1E089E00190E0
:101B50000D928150E1F7109280010BC0E8E5F3E0AF
:101B600080E2819393E0E136F907D9F781E0809331
:101B7000800181E290E09093C6018093C50188E5E1
:101B800093E00E943D1708950F931F938091C50124
:101B90009091C601892BC9F586E090E09093C6012B
:101BA0008093C5018FE097E20E94E5178C018FE0DA
:101BB00097E20E94E5172DB73EB7285030400FB688
:101BC000F8943EBF0FBE2DBFEDB7FEB7319628E5A6
:101BD00033E0ADB7BEB712963C932E93119726E330
:101BE00031E03383228315830483978386830E94A5
:101BF000DF198DE280935C032DB73EB7285F3F4F1E
:101C00000FB6F8943EBF0FBE2DBF88E593E00E944B
:101C10003D171F910F9108958091C5019091C601C4
:101C2000892B11F584E190E09093C6018093C50162
:101C3000EBEAF1E0828193818193919381E0EB3B28
:101C4000F807C1F784E090E00E94E517892B29F49A
:101C50001092BC011092BB0107C00E948C197F73C7
:101C60007093BC016093BB018BEA91E00E94261740
:101C700008958D3011F08A3021F48AE00E945212CA
:101C80008DE00E9452120895CF92DF92EF92FF9260
:101C90000F931F93DF93CF93CDB7DEB7C85CD040CF
:101CA0000FB6F894DEBF0FBECDBF0E94C4128AE704
:101CB0009CE00E945D1281E99CE00E945D1260E858
:101CC00075E280E090E00E9435158AEB9CE00E946E
:101CD000EB1560E875E280E090E00E94F91580E382
:101CE00095E720E931E0F9013197F1F70197D9F74C
:101CF0000E948B0A0E948E130E945B0F0E94AD11FE
:101D00000E945E1782E591E00E94CD0C85EC91E087
:101D10000E94F50E8DEB91E00E94F50E88E0C82E32
:101D200087E0D82E01E07E010894E11CF11C80912F
:101D30007D018330B9F1843028F4813069F182303B
:101D400070F507C08530A1F1853078F18630B1F5A6
:101D500032C08091BD019091BE01892B79F48091B0
:101D600082018F5F80938201843020F00093820192
:101D700010928101D092BE01C092BD01809182017A
:101D8000823069F0833018F48130D1F405C083309B
:101D900049F08430A9F409C00E94220D11C00E94AC
:101DA0000C0E0EC00E94C40D0BC00E94980D08C0FE
:101DB0000E94F70C05C00E94E60C02C00E94D70CDE
:101DC0000E944D12882371F00E943E12182F0E942B
:101DD000390E812FB7010E94AD0C882319F0C7017D
:101DE0000E94660C0E944C09A2CF9C01ADE6B3E0B4
:101DF000E0E0F0E08D919C911197892B41F4EE0F7A
:101E0000FF1FE359FC4F3183208381E00895319611
:101E10001296EC30F10571F780E008959C01ADE673
:101E2000B3E0E0E0F0E08D919C9111978217930769
:101E300041F4EE0FFF1FE359FC4F1182108281E045
:101E4000089531961296EC30F10569F780E0089517
:101E50009C01A4E6B3E0E0E0F0E08D919C91119745
:101E6000892B41F4EE0FFF1FEC59FC4F3183208387
:101E700081E0089531961296E430F10571F780E023
:101E800008959C01A4E6B3E0E0E0F0E08D919C9120
:101E900011978217930741F4EE0FFF1FEC59FC4F87
:101EA0001182108281E0089531961296E430F10596
:101EB00069F780E008953B9A84B5826084BD8FEC19
:101EC00087BD16BCEEE6F0E080818260808385B538
:101ED000846085BD789408951F920F920FB60F927B
:101EE00011242F933F934F935F936F937F938F931F
:101EF0009F93AF93BF93EF93FF93909183019230A1
:101F000030F48FEC87BD9F5F909383018DC080ED8F
:101F100087BD109283018091880390918903019677
:101F20009093890380938803809185039091860321
:101F300001969093860380938503ADE6B3E0ED911F
:101F4000FC911197309749F080819181892B29F07C
:101F500080819181019791838083129683E0A538D7
:101F6000B80769F780916C038F5F80936C03809151
:101F70006C03843611F410926C03809184018F5F9E
:101F800080938401843661F58091620390916303AC
:101F90000196909363038093620310928401809171
:101FA00087038F5F80938703809187038C33C1F40D
:101FB0001092870380918A038F5F80938A038091B8
:101FC0008A038C3369F410928A0380918B038F5FAC
:101FD00080938B0380918B03883111F410928B03D3
:101FE0008091870380FF1DC0439AE0916403F091C4
:101FF0006503309709F00995E0916603F091670356
:10200000309709F00995E0916803F09169033097E2
:1020100009F00995E0916A03F0916B03309719F488
:1020200003C04398E2CF0995FF91EF91BF91AF9123
:102030009F918F917F916F915F914F913F912F91E0
:102040000F900FBE0F901F90189590939903809357
:102050009803089510929903109298030895AC0183
:1020600020E030E0F901EB57FE4FDA01A20FB31F79
:102070008D919C91918380832E5F3F4F2C30310551
:1020800089F70895109286011092850110928801B7
:102090001092870110928A011092890110928C018E
:1020A00010928B0110928E0110928D01109290016E
:1020B00010928F0108951092910181E08093920116
:1020C000089581E0809392010895109292011092F8
:1020D000A7031092A603E0919803F091990330971B
:1020E00009F009950895982F80919501981710F49B
:1020F000909391010895EF92FF920F931F93CF93C6
:10210000DF937C0187E0689F800111240F5F1F4FE0
:10211000C0E0D0E0CE018F5F282FF801EE0FFF1F47
:10212000EE0DFF1D85919491FE01EE0FFF1FE65607
:10213000FC4F91838083808191818F5F9F4F29F431
:10214000822F6FEF7FEF0E94011321960F5F1F4FC9
:10215000C630D105F9F6DF91CF911F910F91FF9015
:10216000EF900895FF920F931F93CF93DF93809189
:102170009201882309F4C2C0809193019091940147
:10218000892B09F4BBC005E811E0C0E0D0E0FF24D2
:10219000F394F80140815181CE01880F991FDC0131
:1021A000A656BC4F2D913C911197FC01E457FC4F72
:1021B00080819181281B390BB1F14115510529F01E
:1021C000808191818F5F9F4F69F4FE01EE0FFF1FA9
:1021D000DF01A656BC4F8D919C91E457FC4F918333
:1021E00080831CC01216130644F4421753076CF484
:1021F00080819181840F951F0AC0241735072CF424
:1022000080819181841B950B02C08D919C9191835B
:102210008083FE01EE0FFF1FE457FC4F6081718148
:102220008F2D0E9401132196F3940E5F1F4F87E0BC
:10223000F81609F0AECF8091A6039091A703892BE1
:1022400009F05CC07091910160919501272F30E0F9
:10225000862F90E0019740919301509194012817A7
:102260003907D4F4CA01672F0E947B108091910135
:102270002EE0829F90011124E0919301F09194014E
:10228000E20FF31F259134913093A7032093A60307
:102290008F5F8093910132C01EE0619FF001112495
:1022A0003E97E40FF51F859194916150892B79F445
:1022B000CA010E947B101092920110929101E0914C
:1022C0009803F09199033097C9F0099517C0CA0196
:1022D0000E947B1080919501819FC00111240E976F
:1022E000E0919301F0919401E80FF91F8591949189
:1022F0009093A7038093A60310929101DF91CF9151
:102300001F910F91FF900895CF93DF931092920148
:1023100010929101909394018093930160939501A1
:10232000C0E0D0E09E012F5F822F0E942813FE01A3
:10233000EE0FFF1FDF01A457BC4F11969C938E93A5
:102340008D919C91E656FC4F918380832196C630F7
:10235000D10541F7DF91CF91089582EB90E10E9482
:10236000280F86EA93E00E94F50E0895E1ECF0E074
:102370008081806880830895E1ECF0E080818F7730
:10238000808308951F920F920FB60F9211242F93FE
:102390008F939F93EF93FF932091C6009091F0034A
:1023A0008091F1039817D8F4E091F403F091F503CC
:1023B00021938091F703815021F48091F103E81B70
:1023C000F1098093F703F093F503E093F4039FB7CB
:1023D000F8948091F0038F5F8093F0039FBFFF918B
:1023E000EF919F918F912F910F900FBE0F901F90A3
:1023F00018951F920F920FB60F9211242F938F935F
:102400009F93EF93FF938091E8038823F1F0E0918D
:10241000EA03F091EB0321918091EE03815021F4C6
:102420008091E903E81BF109F093EB03E093EA03E1
:102430008093EE039FB7F8948091E80381508093D6
:10244000E8039FBF2093C60005C08091C1008F7D27
:102450008093C100FF91EF919F918F912F910F90E9
:102460000FBE0F901F90189580EF93E00E94C00A56
:10247000089580EF93E00E94D80A089580EF93E0DA
:102480000E94D80A089588EE93E00E94F40A20E0A2
:10249000892B09F421E0822F089580EF93E00E94B8
:1024A000F40A0895682F88EE93E00E94A50AE1ECF3
:1024B000F0E09081906290830895CF93DF93EC01D8
:1024C00002C00E945212FE01219684918823C9F70E
:1024D000DF91CF9108951F93CF93DF93EC0110E02C
:1024E00003C00E9452121F5FFE01E10FF11D8081A7
:1024F000882311F01F3FA9F7DF91CF911F91089515
:102500001F931FB79C0140E050E084E0220F331F6F
:10251000441F551F8A95D1F760E074E284EF90E084
:102520000E948718215030403093C5002093C4008A
:10253000F8941092C00088E98093C10086E08093EF
:10254000C2008091C6008091C00087FDFACF80EC68
:102550008093C0001FBF789480EF93E068EA73E037
:1025600040E40E949B0A88EE93E068EF73E04FEF2F
:102570000E949B0A1F91089580E895E20E948012B4
:1025800084E28093C200089580E895E20E94801260
:10259000089586E08093960180E29EE49093850002
:1025A00080938400EFE6F0E08081816080837894FE
:1025B000E1E8F0E08081826080830895CF93DF932B
:1025C000A1E2B5E0C4E1D5E041E050E0ED91FD913C
:1025D0002081CA01099002C0880F991F0A94E2F76E
:1025E00080958223808385E0AD32B80779F78091AA
:1025F0006F008E7F80936F0010928100DF91CF91EA
:102600000895E82F8150863010F577FF0AC0F0E07A
:10261000EE0FFF1FEB50FB4F8FEF9FEF91838083F7
:10262000089589E0653C78071CF064EC79E006C009
:1026300081E0643F780714F464EF71E0F0E0EE0F9E
:10264000FF1FEB50FB4F660F771F71836083089568
:10265000E82F8150863018F0E0E0F0E011C0F0E0A3
:10266000EE0FFF1FEB50FB4F808191812FEF8F3FCB
:10267000920719F4EFEFFFEF03C0FC01F695E79521
:10268000CF010895809120058A3048F08FEF9FEFA9
:1026900090933D0580933C052FEF3FEF1CC0809148
:1026A00020058823A1F480910F05882381F0809173
:1026B0003A0590913B0562E070E00E9474189B011E
:1026C00070933D0560933C0510920F0504C0209166
:1026D0003C0530913D05C901089580B78B7F80BFCF
:1026E000E1E8F0E080818F778083EFE6F0E08081A1
:1026F0008F7D8083209810921305109212051092FE
:1027000011051092100510923905109220058FEFD7
:102710009FEF90933D0580933C050895EF92FF92C3
:102720000F931F93CF93DF93E7EFF4E08FEF9FEFCB
:102730008193919325E0EF30F207D1F72BE230E05F
:1027400030932205209321053093240520932305FF
:1027500030932605209325053093280520932705DF
:1027600085E290E090932A058093290590932C05AB
:1027700080932B0530932E0520932D0590933005E3
:1027800080932F0590933205809331059093340503
:1027900080933305909336058093350590933805E3
:1027A0008093370582E08093140594E0909315059B
:1027B00025E02093160586E08093170581E080933D
:1027C000180583E08093190580931A0590931B05E3
:1027D00090931C0520931D058BE080931E058CE0D3
:1027E00080931F05C1E2D5E044E155E0DE01BA0166
:1027F00001E010E0ED90FD90F7012081FB01C801A0
:10280000019002C0880F991F0A94E2F7BF018095DA
:102810008223F7018083F5E0AD32BF0759F761E00D
:1028200070E0E991F9912291DA01CB010D9002C09B
:10283000880F991F0A94E2F7AD01282B2083B5E099
:10284000CD32DB0771F780916F008E7F80936F0030
:1028500086E0809396011092800080E29EE490933F
:102860008500809384000E946D130E94C912DF913D
:10287000CF911F910F91FF90EF900895E1E8F0E064
:10288000808180648083B59A10923905EFE6F0E08C
:10289000808180628083089580916F008F7D809316
:1028A0006F00809139058823A1F010922005809156
:1028B0001005909111052091120530911305821B8E
:1028C000930B90933B0580933A0581E080930F052D
:1028D0000895809120058B3028F4809120058F5F2A
:1028E0008093200508951F920F920FB60F92112426
:1028F0002F933F934F935F936F937F938F939F9308
:10290000AF93BF93EF93FF9380919601863028F0A9
:102910000E944C14109296011FC0E0919601F0E0C5
:10292000EE0FFF1FEF5DFA4FA081B1812C91E09176
:102930009601F0E0EC5EFA4F81E090E0008002C08A
:10294000880F991F0A94E2F7809582238C938091D7
:1029500096018F5F8093960180919601863048F0B2
:1029600080E29EE490938500809384000E943E1450
:1029700038C0E0919601F0E0EE0FFF1FE950FB4FE9
:10298000808191818F5F9F4F31F1E0919601F0E05E
:10299000EE0FFF1FEF5DFA4FA081B1812C91E09106
:1029A0009601F0E0EC5EFA4F81E090E0008002C01A
:1029B000880F991F0A94E2F7282B2C93E091960137
:1029C000F0E0EE0FFF1FE950FB4F80819181909561
:1029D00081959F4F02C08CE09EEF9093850080937D
:1029E0008400FF91EF91BF91AF919F918F917F9163
:1029F0006F915F914F913F912F910F900FBE0F906C
:102A00001F9018951F920F920FB60F9211248F935B
:102A10009F93F8948091810086FF0FC0809186007B
:102A20009091870090931305809312058091810007
:102A30008F7B80938100B59A10C080918600909121
:102A40008700909311058093100581E080933905EC
:102A500080916F008F7D80936F0078949F918F910C
:102A60000F900FBE0F901F901895EF92FF920F934B
:102A70001F93CF93DF937B018C01109298011092EA
:102A8000970110929A011092990110929C01109254
:102A90009B0110929E0110929D01389A409A20E06D
:102AA00030E0E901CC0FDD1FC20FD31FBE01660F5E
:102AB000771F660F771FAB01425E504FFA01859179
:102AC0009591A591B4918E159F05A007B10729F5A1
:102AD000FB01EE5DF04F8591949190939801809366
:102AE0009701FB01EC5DF04F8591949190939A01D1
:102AF00080939901FB01EA5DF04F85919491909349
:102B00009C0180939B01FB01E85DF04F85919491BE
:102B100090939E0180939D0106C02F5F3F4F2C3004
:102B2000310509F0BECFDF91CF911F910F91FF903A
:102B3000EF900895F82F20919D0130919E0121156D
:102B4000310509F432C0EFB7F894409888B12B5F93
:102B50003F4FC90140E001974FEF8F3F9407D9F7EE
:102B60002550304051E060E070E0A0E0852F8F23D9
:102B700011F0409A01C0409888B1C9014A2F0197CD
:102B80004FEF8F3F9407D9F7550F6F5F7F4F683036
:102B9000710561F7409A88B1EFBF7894C90120E0D0
:102BA00001972FEF8F3F9207D9F708951F93CF9387
:102BB000DF93EC0110E003C00E949A151F5FFE0135
:102BC000E10FF11D8081882311F01F3FA9F7DF91EC
:102BD000CF911F910895CF93DF93EC0102C00E9423
:102BE0009A15FE01219684918823C9F7DF91CF9130
:102BF0000895EF92FF920F931F93CF93DF937B0182
:102C00008C011092A00110929F011092A2011092CB
:102C1000A1011092A4011092A3011092A60110929A
:102C2000A5013C9A449A20E030E0E901CC0FDD1F79
:102C3000C20FD31FBE01660F771F660F771FAB0150
:102C4000425E504FFA0185919591A591B4918E15F0
:102C50009F05A007B10729F5FB01EE5DF04F8591B7
:102C600094919093A00180939F01FB01EC5DF04F44
:102C7000859194919093A2018093A101FB01EA5D5B
:102C8000F04F859194919093A4018093A301FB014F
:102C9000E85DF04F859194919093A6018093A501F2
:102CA00006C02F5F3F4F2C30310509F0BECFDF91BA
:102CB000CF911F910F91FF90EF900895F82F2091E1
:102CC000A5013091A6012115310509F432C0EFB7F5
:102CD000F894449888B12B5F3F4FC90140E00197B9
:102CE0004FEF8F3F9407D9F72550304051E060E017
:102CF00070E0A0E0852F8F2311F0449A01C0449822
:102D000088B1C9014A2F01974FEF8F3F9407D9F738
:102D1000550F6F5F7F4F6830710561F7449A88B136
:102D2000EFBF7894C90120E001972FEF8F3F920702
:102D3000D9F708951F93CF93DF93EC0110E003C000
:102D40000E945E161F5FFE01E10FF11D8081882346
:102D500011F01F3FA9F7DF91CF911F910895CF93F5
:102D6000DF93EC0102C00E945E16FE012196849161
:102D70008823C9F7DF91CF9108958091B40000B600
:102D800005FE05C0439A843630F48F5F04C0439833
:102D9000823008F081508093B4000895892B11F09F
:102DA0002A9801C02A9A80E5982F9A95F1F72D98D4
:102DB00090EA9A95F1F72D9A8A95F1F7089580E5B2
:102DC0008A95F1F72C9880EA8A95F1F72C9A089564
:102DD000EF92FF920F931F93CF93DF937B01CFE08E
:102DE000D0E0082F10E080E090E0C017D10711F488
:102DF00081E090E00E94CE1621978FEFCF3FD80759
:102E000091F7C0E0D0E0C7010C2E02C0880F991FD7
:102E10000A94E2F7807090780E94CE162196C03115
:102E2000D10589F70E94DF16DF91CF911F910F9195
:102E3000FF90EF900895E62FF0E0EE0FFF1FE259AC
:102E4000F04F659174910E94E81608951F931091B8
:102E5000A701E12FF0E0EE0FFF1FE80FF91F6081DF
:102E60007181812F0E94E8161F5F1093A70119300E
:102E700010F01092A7011F9108951F93CF93DF9335
:102E8000EC01FC0101900020E9F73197E81BF90BF8
:102E90001091A8011E1730F4C10FD11D812F688138
:102EA0000E941B17812F8F5F8093A801893011F436
:102EB0001092A801DF91CF911F910895E0EBF0E00F
:102EC0008BE08083808180628083E1EBF0E082E0B0
:102ED000808380818860808388E78093B3008AE064
:102EE0008093B400229A249A259A539A80B78064DA
:102EF00080BFEFE7F0E08081826080838DEB96E118
:102F00000E94280F08952F923F924F925F926F92E6
:102F10007F928F929F92AF92BF92CF92DF92EF9269
:102F2000FF920F931F93DF93CF93CDB7DEB73B0193
:102F30004C0119012A016D897E898F89988D6A1942
:102F40007B098C099D09621A730A840A950AA401F7
:102F500093010E945518E218F30804091509A80105
:102F600097010E94A9182A0D3B1D4C1D5D1DB9013A
:102F7000CA01CF91DF911F910F91FF90EF90DF90E9
:102F8000CF90BF90AF909F908F907F906F905F9009
:102F90004F903F902F9008950F931F93021B130B98
:102FA000861B970B461B570BBC01069FC001079F52
:102FB000900D169F900D1124BA010E947418620F93
:102FC000731FCB011F910F910895CF93DF93EC01F5
:102FD000009719F420E030E006C00E942919BE01D4
:102FE0000E9474189C01C901DF91CF910895CF937D
:102FF000DF93EC01861797073CF4CB018C1B9D0BEC
:103000000E94E517C80FD91FCE01DF91CF91089517
:10301000009711F00E942E190895EF92FF920F93DE
:103020001F937B018C01611571058105910529F4C0
:1030300020E030E040E050E00BC00E948C19A80175
:1030400097010E94A918AC01CB01DA019C01AD01E6
:10305000B901CA011F910F91FF90EF900895EF926F
:10306000FF920F931F937B018C01621773078407F4
:10307000950764F4261B370B480B590BCA01B9019D
:103080000E940D18E60EF71E081F191FB701C80190
:103090001F910F91FF90EF900895611571058105C3
:1030A000910511F00E9491190895629FD001739FBC
:1030B000F001829FE00DF11D649FE00DF11D929FD4
:1030C000F00D839FF00D749FF00D659FF00D992713
:1030D000729FB00DE11DF91F639FB00DE11DF91F37
:1030E000BD01CF011124089597FB092E07260AD0B0
:1030F00077FD04D049D006D000201AF47095619570
:103100007F4F0895F6F7909581959F4F0895A1E21E
:103110001A2EAA1BBB1BFD010DC0AA1FBB1FEE1F51
:10312000FF1FA217B307E407F50720F0A21BB30B9C
:10313000E40BF50B661F771F881F991F1A9469F718
:1031400060957095809590959B01AC01BD01CF0174
:10315000089597FB092E05260ED057FD04D0D7DF22
:103160000AD0001C38F450954095309521953F4F7A
:103170004F4F5F4F0895F6F7909580957095619544
:103180007F4F8F4F9F4F0895AA1BBB1B51E107C074
:10319000AA1FBB1FA617B70710F0A61BB70B881FE7
:1031A000991F5A95A9F780959095BC01CD01089576
:1031B000A0E0B0E0EEEDF8E10C94881CEC01A880F2
:1031C000B980CA80DB80A114B104C104D10441F4E8
:1031D00084E2A82E89EDB82E8BE5C82E87E0D82E84
:1031E000C601B5012DE133EF41E050E00E94A9187E
:1031F00027EA31E440E050E00E9455187B018C0141
:10320000C601B5012DE133EF41E050E00E94A9185D
:10321000CA01B9012CEE34EF4FEF5FEF0E94551851
:103220006E0D7F1D801F911F97FF04C0615070407D
:1032300080409048688379838A839B839B013F7792
:10324000C901CDB7DEB7EAE00C94A41C0E94D818DF
:10325000089580E691E00E94D8180895A0E0B0E0BB
:103260008093600190936101A0936201B093630128
:103270000895A0E0B0E0EFE3F9E10C94881CEC01C4
:10328000A880B980CA80DB80A114B104C104D10434
:1032900041F484E2A82E89EDB82E8BE5C82E87E094
:1032A000D82EC601B5012DE133EF41E050E00E9478
:1032B000A91827EA31E440E050E00E9455187B014C
:1032C0008C01C601B5012DE133EF41E050E00E94D1
:1032D000A918CA01B9012CEE34EF4FEF5FEF0E943D
:1032E00055186E0D7F1D801F911F97FF04C0615000
:1032F000704080409048688379838A839B839B01D8
:10330000AC015F77B901CA01CDB7DEB7EAE00C9432
:10331000A41C0E943919089584E691E00E9439198D
:1033200008956093640170936501809366019093A2
:1033300067010895FC0188279927E894219120329C
:10334000E9F3293010F02E30C8F32B3241F02D3242
:1033500039F4689404C00E94D719820F911D2191FD
:1033600020532A30C0F31EF4909581959F4F089505
:10337000FB01DC018D91019080190110D9F3990BAB
:103380000895FB01DC0101900D920020E1F7089502
:10339000FB01DC014150504048F001900D920020AB
:1033A000C9F701C01D9241505040E0F708957AE0FE
:1033B000979F902D879F802D910D11240895AEE049
:1033C000B0E0E5EEF9E10C948E1C0D891E8986E0D3
:1033D0008C831A8309838FEF9FE79E838D839E01E1
:1033E000275E3F4FCE0101966F89788DA9010E941B
:1033F000031A2F813885020F131FF80110822E96B1
:10340000E4E00C94AA1CABE0B0E0E9E0FAE10C9433
:10341000801C3C012B015A01FC011782168283811A
:1034200081FD03C06FEF7FEFC6C19AE0892E1E01B8
:103430000894211C311CF3012381F20123FD8591A5
:1034400023FF81912F01882309F4B2C1853239F419
:1034500023FD859123FF81912F01853229F490E08E
:10346000B3010E94F61BE7CF982FFF24EE24992486
:10347000FFE1FF15D0F09B3269F09C3228F49032C6
:1034800059F0933291F40EC09D3249F0903369F4B3
:1034900041E024C052E0F52A84E0F82A28C098E0F0
:1034A000F92A25C0E0E1FE2A22C0F7FC29C0892FB5
:1034B00080538A3070F4F6FE05C0989C902C11243D
:1034C000980E15C0E89CE02C1124E80EF0E2FF2ACB
:1034D0000EC09E3229F4F6FC6BC140E4F42A07C00A
:1034E0009C3619F450E8F52A02C0983649F4F201E6
:1034F00023FD959123FF91912F01992309F0B8CFD6
:10350000892F8554833018F08052833038F444E09A
:1035100050E0A40EB51E5FE359830FC0933631F01F
:10352000933779F0933509F056C020C0F5018081BA
:10353000898342E050E0A40EB51E610101E010E075
:1035400012C0F501C080D180F6FC03C06FEF7FEFA1
:1035500002C0692D70E042E050E0A40EB51EC60125
:103560000E94EB1B8C015FE7F52214C0F501C080BF
:10357000D180F6FC03C06FEF7FEF02C0692D70E0D1
:1035800042E050E0A40EB51EC6010E94E01B8C0173
:1035900050E8F52AF3FE07C01AC080E290E0B301BC
:1035A0000E94F61BEA948E2D90E008171907A8F3E5
:1035B0000EC0F601F7FC8591F7FE81916F0190E056
:1035C000B3010E94F61BE110EA940150104001156E
:1035D000110579F7EAC0943611F0993669F5F7FECE
:1035E00008C0F501208131814281538184E090E05F
:1035F0000AC0F501808191819C01442737FD4095E7
:10360000542F82E090E0A80EB91E9FE6F92257FFE2
:1036100009C050954095309521953F4F4F4F5F4FD2
:10362000E0E8FE2ACA01B901A1012AE030E00E94C7
:10363000221CD82ED21840C0953729F41F2D1F7E8A
:103640002AE030E01DC01F2D197F9F3661F09037B2
:1036500020F4983509F0ACC00FC0903739F0983796
:1036600009F0A6C004C028E030E00AC0106114FDD3
:10367000146020E130E004C014FD166020E132E067
:1036800017FF08C0F501608171818281938144E058
:1036900050E008C0F50180819181BC0180E090E09C
:1036A00042E050E0A40EB51EA1010E94221CD82EBB
:1036B000D2188FE7F82EF122F6FE0BC05EEFF5224E
:1036C000D91438F4F4FE07C0F2FC05C08FEEF822DE
:1036D00002C01D2D01C0192DF4FE0DC0FE01ED0D1F
:1036E000F11D8081803319F499EEF92208C01F5F23
:1036F000F2FE05C003C08F2D867809F01F5F0F2DE5
:10370000F3FC14C0F0FE0FC01E1510F09D2C0BC072
:103710009D2C9E0C911A1E2D06C080E290E0B301F4
:103720000E94F61B1F5F1E15C0F304C01E1510F487
:10373000E11A01C0EE2404FF0FC080E390E0B30162
:103740000E94F61B02FF1DC001FD03C088E790E048
:103750000EC088E590E00BC0802F867891F001FFC5
:1037600002C08BE201C080E2F7FC8DE290E0B30181
:103770000E94F61B06C080E390E0B3010E94F61B96
:103780009A94D914C0F3DA94F101ED0DF11D808102
:1037900090E0B3010E94F61BDD20A9F706C080E28D
:1037A00090E0B3010E94F61BEA94EE20C1F743CEED
:1037B000F30166817781CB012B96E2E10C949C1C8E
:1037C000FC010590615070400110D8F780959095EC
:1037D0008E0F9F1F0895FC016150704001900110F1
:1037E000D8F7809590958E0F9F1F08950F931F9384
:1037F000CF93DF938C01EB018B8181FF1BC082FF94
:103800000DC02E813F818C819D812817390764F47A
:10381000E881F9810193F983E88306C0E885F98599
:10382000802F0995892B31F48E819F8101969F838A
:103830008E8302C00FEF1FEFC801DF91CF911F9160
:103840000F910895FA01AA27283051F1203181F112
:10385000E8946F936E7F6E5F7F4F8F4F9F4FAF4F98
:10386000B1E03ED0B4E03CD0670F781F891F9A1FAB
:10387000A11D680F791F8A1F911DA11D6A0F711D5F
:10388000811D911DA11D20D009F468943F912AE06B
:10389000269F11243019305D3193DEF6CF01089553
:1038A000462F4770405D4193B3E00FD0C9F7F6CF84
:1038B000462F4F70405D4A3318F0495D31FD40524C
:1038C000419302D0A9F7EACFB4E0A69597958795E2
:1038D00077956795BA95C9F70097610571050895C1
:1038E0009B01AC010A2E069457954795379527956D
:1038F000BA95C9F7620F731F841F951FA01D089505
:103900002F923F924F925F926F927F928F929F92EF
:10391000AF92BF92CF92DF92EF92FF920F931F93DD
:10392000CF93DF93CDB7DEB7CA1BDB0B0FB6F8948E
:10393000DEBF0FBECDBF09942A88398848885F84CE
:103940006E847D848C849B84AA84B984C884DF803F
:10395000EE80FD800C811B81AA81B981CE0FD11D23
:103960000FB6F894DEBF0FBECDBFED010895F894F9
:02397000FFCF87
:1039720032131207040319191919300031003200E9
:103982003300340035003600370038003900247324
:103992000024520024253164253264002044414E23
:1039A20047455221200025346420253464000F004D
:1039B2000F000F000F000F000900090009000900A5
:1039C200090044524F494420302E37383600050052
:0839D2000100000001000000EB
:00000001FF
